:020000020000FC
:100000000C94BB1D1895189518951895189518956A
:100010001895189518951895189518951895189578
:100020001895189518951895189518951895189568
:100030001895189518951895189518951895189558
:100040001895189518951895189518951895189548
:100050000C94860518951895189518951895189567
:10006000189518950C945309189518951895189586
:100070001895189518951895189518951895189518
:100080001895189518951895189518951895189508
:1000900018951895189518951895189518951895F8
:1000A00018951895189518951895189518951895E8
:1000B00018951895189518951895189518951895D8
:1000C00018951895189518951895189518951895C8
:1000D00018951895189518951895189518951895B8
:1000E00018951895189518951895189518951895A8
:1000F0001895189518951895189518951895189598
:100100001895189518951895189518951895189587
:100110001895189518951895189518950C947505B7
:100120001895189518951895189518951895189567
:10013000189518950C94F704189518951895189516
:100140001895189518951895189518951895189547
:100150001895189518951895189518951895189537
:100160001895189518951895189518951895189527
:100170001895189518951895189518951895189517
:100180001895189518951895189518951895189507
:1001900018951895189518951895189518951895F7
:1001A00018951895189518951895189518951895E7
:1001B00018951895189518951895189518951895D7
:1001C00018951895189518951895189518951895C7
:1001D00018951895189518951895189518951895B7
:1001E00018951895189518951895189518951895A7
:1001F000189518951895189518951895AA594EBEE2
:1002000034D514BEAE16863CF81D473E59298B3EA8
:10021000F81D473EAE16863C34D514BEAA594EBED4
:10022000D4D26FBCBB3CF2BC872453BD1A6DA4BDB5
:10023000AE76E6BD17740FBEB5875B3F17740FBE71
:10024000AE76E6BD1A6DA4BD872453BDBB3CF2BC9F
:10025000D4D26FBC14BEA1BD6FEDFCBDDC252FBE9A
:10026000E9383F3FDC252FBE6FEDFCBD14BEA1BDBC
:10027000010102040804040201012A2A2A2A2A2A66
:030280002A2A2AFD
:1002840000017F247E2445532402462411BF230BFE
:10029400842301D82301532401512401462402D884
:1002A4002305712301B22301BF23038D2302BF233E
:1002B40003BB23FB0BEC0093520008E000935000B7
:1002C400E1E5F0E0008103FFFBCF03EC0093550070
:1002D400E0E5F0E0008100610083E1E5F0E0008109
:1002E40004FFFBCF08ED04BF04E000934000E0E509
:1002F400F0E000810E7F0083089501E0009328025E
:1003040000E300932902089501E00093300208E31A
:100314000093310208950DE00093200300E400935C
:10032400210300E00093220300E40093240300EE81
:100334000093280300EE00932A0300EE00932A039F
:1003440008950150104098018901232BD1F7089595
:100354008A93802F03C008EE1DEFF3DF8A95082FE0
:10036400802F0023C1F7899108950E94392180E0EC
:1003740090E0A0E0B0E048E0442E1BC0442D50E0E3
:10038400440F551F440F551FFA01E658FE4D0080D7
:10039400118022803380442D50E0440F551F440FB8
:1003A400551FFA01E258FE4D0082118222823382E7
:1003B4004A9441E0441610F7EEE7F1E2008311831A
:1003C40022833383442423C0042D10E0000F111F23
:1003D400000F111FF801E450FE4F459155916591AE
:1003E4007491042D10E0000F111F000F111FF8016C
:1003F400E258FE4D00811181228133810E94BE1F8B
:10040400AC01BD010E945D1FC801D901439409E0FC
:100414004016D0F28C019D01E5E00C944A210E9423
:10042400392180E090E0A0E0B0E048E0442E1BC019
:10043400442D50E0440F551F440F551FFA01E25656
:10044400FE4D0080118022803380442D50E0440F03
:10045400551F440F551FFA01EE55FE4D00821182BF
:10046400228233824A9441E0441610F7E2EAF1E230
:100474000083118322833383442423C0042D10E09A
:10048400000F111F000F111FF801E450FE4F45919A
:10049400559165917491042D10E0000F111F000F08
:1004A400111FF801EE55FE4D008111812281338127
:1004B4000E94BE1FAC01BD010E945D1FC801D9018D
:1004C400439409E04016D0F28C019D01E5E00C94C0
:1004D4004A210E94392180E090E0A0E0B0E04CE0A5
:1004E400442E1BC0442D50E0440F551F440F551F8C
:1004F400FA01EE53FE4D0080118022803380442D9A
:1005040050E0440F551F440F551FFA01EA53FE4DA6
:1005140000821182228233824A9441E0441610F709
:10052400E6ECF1E20083118322833383442423C065
:10053400042D10E0000F111F000F111FF801E05EE1
:10054400FD4F4591559165917491042D10E0000F74
:10055400111F000F111FF801EA53FE4D0081118194
:10056400228133810E94BE1FAC01BD010E945D1F28
:10057400C801D90143940DE04016D0F28C019D01CD
:10058400E5E00C944A210E94392180E090E0A0E04B
:10059400B0E04CE0442E1BC0442D50E0440F551FE6
:1005A400440F551FFA01EA50FE4D0080118022804D
:1005B4003380442D50E0440F551F440F551FFA015A
:1005C400E650FE4D00821182228233824A9441E039
:1005D400441610F7EAEFF1E2008311832283338398
:1005E400442423C0042D10E0000F111F000F111F1D
:1005F400F801E05EFD4F4591559165917491042D8C
:1006040010E0000F111F000F111FF801E650FE4DFE
:1006140000811181228133810E94BE1FAC01BD0182
:100624000E945D1FC801D90143940DE04016D0F229
:100634008C019D01E5E00C944A210E94392180E05F
:1006440090E0A0E0B0E046E0442E1BC0442D50E012
:10065400440F551F440F551FFA01E65DFD4D008000
:10066400118022803380442D50E0440F551F440FE5
:10067400551FFA01E25DFD4D008211822282338210
:100684004A9441E0441610F7EEE2F2E2008311834B
:1006940022833383442423C0042D10E0000F111F50
:1006A400000F111FF801EC5AFD4F459155916591CA
:1006B4007491042D10E0000F111F000F111FF80199
:1006C400E25DFD4D00811181228133810E94BE1FB4
:1006D400AC01BD010E945D1FC801D901439407E02C
:1006E4004016D0F28C019D01E5E00C944A210E9451
:1006F400392180E090E0A0E0B0E046E0442E1BC049
:10070400442D50E0440F551F440F551FFA01EA5B76
:10071400FD4D0080118022803380442D50E0440F31
:10072400551F440F551FFA01E65BFD4D00821182EF
:10073400228233824A9441E0441610F7EAE4F2E25A
:100744000083118322833383442423C0042D10E0C7
:10075400000F111F000F111FF801EC5AFD4F4591B6
:10076400559165917491042D10E0000F111F000F35
:10077400111FF801E65BFD4D008111812281338157
:100784000E94BE1FAC01BD010E945D1FC801D901BA
:10079400439407E04016D0F28C019D01E5E00C94EF
:1007A4004A219A938A93842F682F70E0660F771FEB
:1007B400660F771FFB01EA59FD4D008011802280EE
:1007C40033800019110922093309052E1124A001CF
:1007D40060E070E00E949C1E482F50E0440F551FBB
:1007E400440F551FFA01EA59FD4D40815181628140
:1007F4007381040F151F261F371F90E0880F991F60
:10080400880F991FFC01EA59FD4D0083118322834F
:1008140033838991999108951091480001E00093E0
:1008240048002091A0003091A2000091A2000C7F0A
:1008340004600093A2004FB77894E8E4F0E00081EC
:10084400016000835091CD01EF93FF930F932F9399
:10085400EBECF1E008ED21E004BF20832F910F9130
:10086400FF91EF9103E00093CD0188951093480028
:100874002093A0003093A2005093CD014FBF089560
:10088400EFECF1E0008107FDFBCF0895F9DFEFEC19
:10089400F1E0008101FF11C006E30093CA01EF9368
:1008A400FF930F932F93EBECF1E008ED21E004BFED
:1008B40020832F910F91FF91EF9108959A938A933A
:1008C400C801DEDFFC01E05CF140B89750F44091D0
:1008D400192450E009E010E00E94091E800F911FC6
:1008E40017C0803901E0900798F44091182450E033
:1008F40000E210E00E94091E98014091192450E082
:1009040000E610E00E94091E200F311F820F931F82
:10091400082F0093C001892F8F718093C10100E0DB
:100924000093C20106E00093CA01EF93FF930F9373
:100934002F93EBECF1E008ED21E004BF20832F912D
:100944000F91FF91EF910091C401899199910895BC
:100954000E943B21C801A22F00E00093060900E099
:1009640000934608FC01E05CF140B89750F44091D4
:10097400192450E009E010E00E94091E800F911F25
:1009840017C0803901E0900798F44091182450E092
:1009940000E210E00E94091E98014091192450E0E1
:1009A40000E610E00E94091E200F311F820F931FE2
:1009B4006DDF03E30093CA01082F0093C001892F60
:1009C4008F718093C10100E00093C201A093C40120
:1009D40005E30093CA0120DF03E00093060901E068
:1009E40000934608E3E00C944C219A938A93FA937B
:1009F400EA930A927A936A935A934A933A932A937C
:100A04001A930A930FB60091E0230395077000939D
:100A1400E0230091E02310E0000F111FF801ED53D3
:100A2400FD4D0081118100933A0310933B03009123
:100A3400E02310E0000F111FF801ED54FD4D00817B
:100A440011810093380310933903E0E0F2E0008150
:100A5400046000830091E2230023B1F10091532349
:100A640010915423212F220F220B322F4091E02387
:100A740050E0440F551F440F551FFA01ED5EFC4D25
:100A84004081518162817381400F511F621F731F26
:100A9400408351836283738380916423909165239F
:100AA40001968093642390936523009166231091AB
:100AB40067238017910741F400E00093E22310E0DC
:100AC40000936423109365230FBE09911991299112
:100AD400399149915991699179910990E991F991E3
:100AE4008991999118952A931A930A932FB7009193
:100AF40010021091110200935323109354232FBF1B
:100B040009911991299118955A924A92BA93AA93E4
:100B14009A938A93FA93EA933A922A921A920A92AD
:100B24007A936A935A934A933A932A931A930A9319
:100B34005FB60091E223002309F09DC38091DC237A
:100B44009091DD2301968093DC239093DD238E31F5
:100B540000E0900719F400E000931B248091DA234D
:100B64009091DB2301968093DA239093DB238037E3
:100B740007E1900749F400E010E00093DA231093B2
:100B8400DB2301E00093FC230091DA230F7701308B
:100B940019F401E00093032480E036C05091E82367
:100BA400482F642F082F10E0000F111F000F111F92
:100BB400F801ED5EFC4D0081118122813381409169
:100BC400E9230E94711E462FECDD482F50E0440FAC
:100BD400551F440F551FFA01ED5CFC4D0083118332
:100BE4002283338300E010E020E030E0482F50E01F
:100BF400440F551F440F551FFA01ED5EFC4D008351
:100C04001183228333838395883040F20FEF00935E
:100C1400E22300E010E020E030E0E4E7F3E20083C8
:100C2400118322833383E0E7F3E200831183228379
:100C3400338300E010E020E030E0E4E1F4E20083FC
:100C4400118322833383442495C0042D10E0000FC4
:100C5400111F000F111FF801ED5CFC4D4081518103
:100C640062817381042D10E0000F111F000F111F0A
:100C7400F801ED5CFC4D00811181228133810E94D9
:100C8400491E0E94FE1EE4E1F4E24081518162812A
:100C940073810E945D1FE4E1F4E2008311832283E7
:100CA4003383E0E7F3E200811181228133810E94E2
:100CB400FE1EC801D901042D10E0000F111F000F02
:100CC400111FF801ED5CFC4D0081118122813381FB
:100CD4000E94FE1E442D50E0440F551F440F551F23
:100CE400FA01ED52FD4D40815181628173810E9470
:100CF400BE1FAC01BD010E945D1F0E940B1FE0E7F7
:100D0400F3E20083118322833383E4E7F3E2008177
:100D14001181228133810E94FE1EC801D901042D54
:100D240010E0000F111F000F111FF801ED5CFC4DC6
:100D340000811181228133810E94FE1E442D50E0E6
:100D4400440F551F440F551FFA01ED50FD4D4081CE
:100D54005181628173810E94BE1FAC01BD010E945A
:100D64005D1F0E940B1FE4E7F3E2008311832283DB
:100D74003383439408E0401608F467CF40E050E022
:100D840060E071E4E4E1F4E20081118122813381C5
:100D94000E9437200E945727E4E1F4E20083118384
:100DA4002283338300916A2310916B2320E030E087
:100DB4000E94091FA801B901E4E1F4E20081118154
:100DC400228133810E9437200E940B1F00936223EB
:100DD400109363230091E92310E0F801EA58FD4FD2
:100DE400449150E000916223109163230E941D1EE0
:100DF40000936223109363230091DE2310E0F80133
:100E0400E059FD4F449150E0009162231091632317
:100E14000E941D1E00936223109363230091DE231E
:100E2400002351F40091622310916323000F111FDA
:100E34000093622310936323E0E7F3E200811181BE
:100E440022813381E0E8F3E2008311832283338338
:100E5400E4E7F3E20081118122813381E4E8F3E2E3
:100E64000083118322833383ECE8F3E20081118150
:100E740022813381E0E8F3E2408151816281738110
:100E840004171507260737077CF4ECE8F3E2008122
:100E94001181228133810F5F1F4F2F4F3F4F0083FA
:100EA4001183228333830EC0ECE8F3E200811181C5
:100EB400228133810150104020403040008311834F
:100EC40022833383E8E8F3E20081118122813381B4
:100ED400E4E8F3E2408151816281738104171507CC
:100EE400260737077CF4E8E8F3E2008111812281C8
:100EF40033810F5F1F4F2F4F3F4F00831183228396
:100F040033830EC0E8E8F3E200811181228133814A
:100F140001501040204030400083118322833383EA
:100F24000091E1230023D9F000E00093E123E0E8FD
:100F3400F3E20081118122813381ECE8F3E2008342
:100F4400118322833383E4E8F3E200811181228157
:100F54003381E8E8F3E20083118322833383ECE8EE
:100F6400F3E20081118122813381E0E8F3E24081E0
:100F7400518162817381401B510B620B730B40835F
:100F8400518362837383E8E8F3E200811181228153
:100F94003381E4E8F3E24081518162817381401B33
:100FA400510B620B730B4083518362837383E0E8BC
:100FB400F3E20081118122813381E8EBF3E20083C3
:100FC400118322833383E4E8F3E2008111812281D7
:100FD4003381ECEBF3E200831183228333830091AA
:100FE400E423013009F077C00091F323013029F59F
:100FF400E0E8F3E200811181228133810E94FE1E28
:101004000E94B7010E940B1FE8EAF3E200831183F8
:1010140022833383E4E8F3E2008111812281338166
:101024000E94FE1E0E9411020E940B1FECEAF3E2D2
:10103400008311832283338366C00091F32302303B
:1010440029F5E0E8F3E200811181228133810E94D5
:10105400FE1E0E946B020E940B1FE8EAF3E200836B
:10106400118322833383E4E8F3E200811181228136
:1010740033810E94FE1E0E94C5020E940B1FECEAEF
:10108400F3E200831183228333833DC0E0E8F3E27B
:1010940000811181228133810E94FE1E0E941F0360
:1010A4000E940B1FE8EAF3E2008311832283338357
:1010B400E4E8F3E200811181228133810E94FE1E63
:1010C4000E9479030E940B1FECEAF3E20083118370
:1010D4002283338318C0E0E8F3E200811181228186
:1010E4003381E8EAF3E20083118322833383E4E863
:1010F400F3E20081118122813381ECEAF3E200837F
:10110400118322833383E8EAF3E20081118122818F
:101114003381E0EBF3E24081518162817381400FBE
:10112400511F621F731F4083518362837383ECEAF0
:10113400F3E20081118122813381E4EBF3E2408107
:10114400518162817381400F511F621F731F40835D
:10115400518362837383E8EBF3E20081118122817E
:101164003381E0ECF3E24081518162817381400F6D
:10117400511F621F731F4083518362837383ECEB9F
:10118400F3E20081118122813381E4ECF3E24081B6
:10119400518162817381400F511F621F731F40830D
:1011A4005183628373830091F92303950093F92398
:1011B4001091F623101708F05EC000E00093F923A5
:1011C400E0EBF3E20081118122813381E8E7F3E26D
:1011D400008311832283338300E010E020E030E0B9
:1011E400E0EBF3E20083118322833383E4EBF3E245
:1011F4000081118122813381ECE7F3E200831183C2
:101204002283338300E010E020E030E0E4EBF3E2FB
:101214000083118322833383E0ECF3E200811181A4
:1012240022813381E8ECF3E2008311832283338348
:1012340000E010E020E030E0E0ECF3E20083118312
:1012440022833383E4ECF3E2008111812281338130
:10125400ECECF3E2008311832283338300E010E09B
:1012640020E030E0E4ECF3E2008311832283338353
:1012740001E00093EF235FBE0991199129913991FF
:1012840049915991699179910990199029903990CE
:10129400E991F99189919991A991B99149905990BC
:1012A40018954A92BA93AA939A938A93FA93EA93D3
:1012B4003A922A921A920A927A936A935A934A9386
:1012C4003A932A931A930A934FB600E010E00093DE
:1012D4000824109309248091A008813461F4EBE17F
:1012E400F4E200810160008300E010E00093DC235D
:1012F4001093DD2377C500911B24002309F472C5E4
:1013040000911B24033031F400911B24002309F0C5
:1013140019C468C58434F9F401E291D500915723C6
:1013240096D500915F2393D5E8E7F3E2008111811C
:1013340045E00E94171E8BD5ECE7F3E20081118192
:1013440045E00E94171E83D50091012480D500E05A
:1013540000931B24D9CF833571F40091EB230A95B4
:101364000093EB23002319F401E00093EB2300E046
:1013740000931B24C9CF843571F40091EB230395AA
:101384000093EB23053118F004E10093EB2300E014
:1013940000931B24B9CF863471F40091F323039591
:1013A4000093F323043018F001E00093F32300E0EA
:1013B40000931B24A9CF873509F05EC00E94F21464
:1013C40001E23DD597D743D54FE050E00091622329
:1013D400109163230E941D1E3AD50091F32337D543
:1013E4000091EB2334D50091F22331D50091E4230D
:1013F4002ED5009119242BD50091182428D50091BD
:10140400FD2325D5E0915523F09156233196AF0164
:10141400652F660F660B762F00E81DE82BE530E09C
:101424000E949C1E00930E2410930F2400910E24FE
:1014340010910F241A930A9324E231E206EA12E28D
:101444000E943C27229606EA12E2E1D401EF11E061
:1014540035DAFDD400916123FAD40091622310910E
:101464006323083E23E0120718F401E00093E1230C
:1014740000E000931B2448CF853409F06DC00E941E
:10148400F21401E2DCD400911924E1D4009118246F
:10149400DED40091FD23DBD40091E823D8D400915D
:1014A400FA23D5D40091DE23D2D40091E923CFD4FA
:1014B4000091F623CCD40091F423C9D40091E32302
:1014C400C6D40091F523C3D40091EA23C0D400917B
:1014D400EC23BDD40091FF23BAD40091FE23B7D4EA
:1014E400E0915523F09156233196AF01652F660F95
:1014F400660B762F00E81DE82BE530E00E949C1E69
:1015040000930E2410930F2400910E2410910F24A5
:101514001A930A9324E231E206EA12E20E943C277B
:10152400229606EA12E273D4EFE3F1E2008111811C
:10153400228133813A932A931A930A9329E231E25E
:1015440006EA12E20E943C27249606EA12E25FD4DD
:1015540000E000931B24D8CE8B3299F400915C23D5
:1015640076D400915D2373D44FE050E00091622360
:10157400109163230E941D1E6AD400E000931B2473
:10158400C3CE8F3661F406E10E94EE12E4E8F6E081
:1015940000810B7F008300E000931B24B5CE8937C4
:1015A40009F043C001E24BD40091192450D40091B6
:1015B40018244DD40091FD234AD4E0915523F09191
:1015C40056233196AF01652F660F660B762F00E820
:1015D4001DE82BE530E00E949C1E00930E2410931E
:1015E4000F2400910E2410910F241A930A9324E2DD
:1015F40031E206EA12E20E943C27229606EA12E24F
:1016040006D40091D0231091D1231A930A932EE289
:1016140031E206EA12E20E943C27229606EA12E22E
:10162400F6D300E000931B246FCE853741F5E0919B
:101634005523F09156233196AF01652F660F660B43
:10164400762F00E81DE82BE530E00E949C1E0093F5
:101654000E2410930F2400910E2410910F241A933A
:101664000A9324E231E206EA12E20E943C2722961F
:1016740006EA12E2CCD300E000931B2445CE89365F
:1016840031F4F7D5E4D300E000931B243DCE813739
:1016940039F401E00093E42300E000931B2434CEEA
:1016A4008E3639F400E00093E42300E000931B2419
:1016B4002BCE823671F4009144060F7000934406D9
:1016C400E4E6F6E000810D7F008300E000931B2434
:1016D4001BCE803579F408E00093A4080FE00E9443
:1016E400AA0108E10093A4088091A00800E00093F7
:1016F4001B240ACE853649F4009124060360009326
:10170400240600E000931B24FFCD823749F40091A6
:1017140024060C7F0093240600E000931B24F4CDE0
:101724008636C1F5E5E5F3E20081118101501040F0
:1017340000831183009155231091562300932609A9
:1017440010932709E0915523F09156233196AF0168
:10175400652F660F660B762F00E81DE82BE530E059
:101764000E949C1E00930E2410930F2400910E24BB
:1017740010910F241A930A9324E231E206EA12E24A
:101784000E943C27229606EA12E241D300E000932D
:101794001B24BACD8736C1F5E5E5F3E2008111815A
:1017A4000F5F1F4F0083118300915523109156231F
:1017B4000093260910932709E0915523F0915623AD
:1017C4003196AF01652F660F660B762F00E81DE892
:1017D4002BE530E00E949C1E00930E2410930F24EE
:1017E40000910E2410910F241A930A9324E231E2FB
:1017F40006EA12E20E943C27229606EA12E207D386
:1018040000E000931B2480CD883649F5A7D3E091EE
:101814005523F09156233196AF01652F660F660B61
:10182400762F00E81DE82BE530E00E949C1E009313
:101834000E2410930F2400910E2410910F241A9358
:101844000A9324E231E206EA12E20E943C2722963D
:1018540006EA12E2DCD200E000931B2455CD8B365D
:1018640031F5E091D023F091D1233197E093D02347
:10187400F093D123FF2332F408E611E00093D02340
:101884001093D12397D50091D0231091D1231A938B
:101894000A932EE231E206EA12E20E943C272296E3
:1018A40006EA12E2B4D200E000931B242DCD8A365E
:1018B40041F5E091D023F091D1233196E093D023E8
:1018C400F093D123E83601E0F00734F000E010E0B3
:1018D4000093D0231093D1236DD50091D023109180
:1018E400D1231A930A932EE231E206EA12E20E940D
:1018F4003C27229606EA12E28AD200E000931B24D7
:1019040003CD8C36A9F465D30091D0231091D12353
:101914001A930A9323E331E206EA12E20E943C2777
:10192400229606EA12E273D200E000931B24ECCC68
:10193400873759F40E94F2140091FD23023009F410
:1019440091D200E000931B24DFCC843629F508E013
:101954000093E82301E00093FA2305E00093F523C4
:1019640001E00093DE2301E00093E92302E0009309
:10197400F42301E00093F62301E00093E32301E064
:101984000093EA2308E00093EC2308E50093FF2387
:1019940000E000931B24B8CC823579F42FEF0AEFD2
:1019A40011E00E94AA0400E21EE40E94A30108EDD3
:1019B40004BF01E000937900A7CC813339F401E03E
:1019C4000093F02300E000931B249ECC823311F596
:1019D40000E010E00093D8231093D9230093D6237A
:1019E4001093D72320E000E110E00E94AA0420E035
:1019F40001E110E00E94AA042091D8233091D92358
:101A04000091D6231091D7230E942C1500E0009357
:101A14001B247ACC893381F50091FF23039500932D
:101A2400FF230B3518F00AE50093FF230091FF23F1
:101A340010E0119501951040212F220F220B322F17
:101A44000E94FE1E43E353E365E672E40E943720DE
:101A54000E94CC27A801B90100E010E020E83FE390
:101A64000E943720EFE3F1E2008311832283338362
:101A740000E000931B2448CC883381F50091FF23B8
:101A84000A950093FF23063418F406E40093FF2319
:101A94000091FF2310E0119501951040212F220F92
:101AA400220B322F0E94FE1E43E353E365E672E4E9
:101AB4000E9437200E94CC27A801B90100E010E061
:101AC40020E83FE30E943720EFE3F1E20083118333
:101AD4002283338300E000931B2416CC873361F503
:101AE4000ED70BEE11E00E946004B02FA0E00CEEC4
:101AF40011E00E94600410E0A02BB12BA0936E2390
:101B0400B0936F23E0916E23F0916F233196FA9393
:101B1400EA9329E331E206EA12E20E943C27229684
:101B240006EA12E274D103EF11E00E9460048FD13F
:101B340000E000931B24E8CB03E000931B24809374
:101B44001A2450C100911A24063349F4282F0DEEAB
:101B540011E00E94AA0400E000931B2443C10091F9
:101B64001A240533B1F503EF11E00E94600410E07C
:101B740000930E2410930F24E0910E24F0910F246F
:101B8400369734F008ED04BF01E0009379002AC1D0
:101B9400282F0EEE11E00E94AA0422D70091FD2303
:101BA40056D120910E24239503EF11E00E94AA043C
:101BB4002091DA230BEF11E00E94AA040E94D6259B
:101BC400202F0AEE11E00E94AA0400E000931B24D7
:101BD40009C100911A24063531F48093F22300E000
:101BE40000931B24FFC000911A240A3579F48093D2
:101BF40060238091602390E08857904080936A0925
:101C040090936B0900E000931B24ECC000911A240C
:101C1400093481F4803150F48093F5234091F52305
:101C240050E008E710E00E94091EA1D200E00093F2
:101C34001B24D8C000911A24073459F4853028F4A1
:101C44008093DE230091DE23F5D500E000931B246E
:101C5400C9C000911A24003781F48093192420917B
:101C640019240AEF11E00E94AA0400E000931B2447
:101C7400F1D500E000931B24B5C000911A2403376A
:101C840059F580931824282F0DEF11E00E94AA041F
:101C9400882331F40091640608610093640614C03B
:101CA400813059F4E4E6F6E000810F7E0083E4E637
:101CB400F6E000810860008307C0823029F40091B7
:101CC4006406077E0093640600E000931B24C2D5DB
:101CD40000E000931B2486C000911A24083441F4C8
:101CE4008B3010F48093E82300E000931B247AC027
:101CF40000911A24033641F4843010F48093FA23BB
:101D040000E000931B246EC000911A240A3741F4AA
:101D1400833010F48093E92300E000931B2462C015
:101D240000911A240D3441F4843010F48093F62386
:101D340000E000931B2456C000911A24023441F49D
:101D4400853010F48093F42300E000931B244AC0F0
:101D540000911A24013641F4833010F48093E32374
:101D640000E000931B243EC000911A24043759F468
:101D7400873010F48093EA230091EA23A7D700E088
:101D840000931B242FC000911A24083741F48A3091
:101D940010F48093EC2300E000931B2423C00091F3
:101DA4001A240D3661F490E0880F991F8093D02394
:101DB4009093D123FFD200E000931B2413C0009121
:101DC4001A240D3361F48093FE232091FE2305EF42
:101DD40011E00E94AA0400E000931B2403C000E069
:101DE40000931B244FBE099119912991399149916E
:101DF4005991699179910990199029903990E991B3
:101E0400F99189919991A991B991499018950E9454
:101E14003A21C801A0E007C0B0E0FC01EA0FFB1FB3
:101E2400008115D0A395B0E0FC01EA0FFB1F0081EF
:101E3400002311F0AD3080F3E4E00C944B21E1EA8F
:101E4400F8E0108115FFFBCF0093A008089501323C
:101E540009F400E4E1EAF8E0108115FFFBCF0093F8
:101E6400A008089530915623232F01E010E00E942A
:101E7400AA042091552302E010E00E94AA043091A4
:101E8400D123232F05E010E00E94AA042091D0233F
:101E940006E010E00E94AA042091E8230DE110E07E
:101EA4000E94AA042091FA230BE110E00E94AA04E4
:101EB4002091F5230CE010E00E94AA042091DE2377
:101EC40004E110E00E94AA042091E9230EE110E04D
:101ED4000E94AA042091F62303E110E00E94AA04C0
:101EE4002091F42307EF11E00E94AA042091E32338
:101EF4000FE110E00E94AA042091F22306EF11E002
:101F04000E94AA042091602308EF11E00E94AA0411
:101F14002091EA2309E010E00E94AA042091EB2317
:101F240003E010E00E94AA042091EC230CE110E0ED
:101F34000E94AA042091F3230DE010E00E94AA0459
:101F44002091FF2308E010E00E94AA042091E423DA
:101F540002EF11E00E94AA042DD208950E943A21B2
:101F6400A0E0B0E0E4E4F6E000810D7F00838CE4BF
:101F740091E012C080932609909327090CED1FEF7E
:101F84000E94A30176D1A017B10728F4D801809349
:101F940055239093562305968D3E02E0900750F307
:101FA4000091552310915623009326091093270975
:101FB400BED330915623232F01E010E00E94AA04DF
:101FC4002091552302E010E00E94AA04E4E00C945E
:101FD4004B210E94362100916C230E94AA01E4E463
:101FE400F6E000810D7F008380E090E0A0E01DC05A
:101FF400ECE7F3E200811181228133810E94FE1E0D
:10200400A801B9012A013B01E8E7F3E2008111814B
:10201400228133810E94FE1EA201B301E9D0800F08
:10202400911F04E10E94AA01A395A53008F345E09D
:1020340050E08C010E94351EC801E091D023F0913C
:10204400D123E81BF90BE65AFF4FE093D023F0931A
:10205400D1230091D0231091D123093621E0120716
:1020640044F0E0EDF3E20081118108561140008351
:1020740011831091D123112342F4E0EDF3E20081A6
:10208400118108591E4F0083118394D1E8E00C9408
:1020940047210E943A21D80180E090E02AC00DE255
:1020A40010E0AC010E94091EF801EA0FFB1FE8369C
:1020B40001E0F00714F0E856F1408F01212F220FC0
:1020C400220B322F0E94FE1E45E35AEF6EE87CE39A
:1020D4000E94BE1F0E948926AC01440F551F440F65
:1020E400551FFA01ED52FD4D008311832283338382
:1020F4000196883000E0900794F2E4E00C944B21C0
:102104000E943A21D80180E090E02AC00DE210E05C
:10211400AC010E94091EF801EA0FFB1FE83601E03A
:10212400F00714F0E856F1408F01212F220F220B03
:10213400322F0E94FE1E45E35AEF6EE87CE30E94B4
:10214400BE1F0E94B71DAC01440F551F440F551FFD
:10215400FA01ED50FD4D00831183228333830196F0
:10216400883000E0900794F2E4E00C944B210E9444
:102174003621D80180E090E034C08D01212F220F58
:10218400220B322F0E94FE1E280139018C01212FBF
:10219400220F220B322F0E94FE1E4BED5FE069E4FA
:1021A4007FE30E94BE1F0E948926A201B3010E9400
:1021B400BE1F280139018D01212F220F220B322F3E
:1021C4000E94FE1EA201B3010E945D1F0E940B1F0C
:1021D4009C01220F331FF901ED53FD4D0083118340
:1021E4000196883000E0900744F2E8E00C9447211F
:1021F4000E944F1D40E050E064E672E40E94BE1F5E
:102204000E940B1F08950E943621C801D9012A019A
:102214003B01A201B3012A013B010091DF2310E03D
:1022240020E030E00E94091FA801B9018201930156
:102234000E943720AC01BD010E945D1FA201B301C1
:102244000E944F1D40E050E064E672E40E94BE1F0D
:102254000E940B1F0B3520E0120714F00AE510E072
:10226400063A2FEF120714F406EA1FEFE8E00C9485
:1022740047210E943A2180E090E000E0009322028E
:1022840000E00093010204E00E94AA01A0E0B0E093
:1022940019C00EE110E00E94A301E0E0F2E0008129
:1022A4000860008300912B020023E1F301E0009316
:1022B4002B020091120210911302801791070CF463
:1022C400C8011196A43F01E0B0071CF300E100939C
:1022D400010202E000932202835D9040992312F4EC
:1022E40080E090E042E050E08C010E94351EE4E082
:1022F4000C944B21E0E0F2E0008100610083009146
:1023040033020023E1F301E0009333024091EE2312
:1023140050E000911402109115020E941D1E20919C
:10232400F72330E0220F331F220F331F020F131F36
:1023340008950E943A210EE210E0C4D2802F0FE2E9
:1023440010E0C0D2482F502F8A01212F220F220BD8
:10235400322F0E94FE1E40E04093010241E0409370
:102364000202E0E0F2E040814062408340913B029F
:102374004423E1F341E040933B02A801B90100E0AA
:1023840010E02EEA33E40E943720C801D9010091FD
:1023940016021091170220E030E00E94091FAC01E0
:1023A400BD010E94BE1F0E940B1F0C521140E4E0AD
:1023B4000C944B210091D0231091D1236ADE00911B
:1023C400D0231091D1239CDE08950091D023109145
:1023D400D1235FDE0091D0231091D12391DE40916F
:1023E400F52350E008E710E00E94091EC0DE0091CA
:1023F4005523109156230093260910932709089515
:102404009A938A9301E010E00E946004902F80E088
:1024140002E010E00E94600410E0802B912B809376
:1024240055239093562305E010E00E946004902FFA
:1024340080E006E010E00E94600410E0802B912B05
:102444008093D0239093D1230EE010E00E94600487
:10245400902F80E00FE010E00E94600410E0802BD9
:10246400912B8093D6239093D72300E110E00E9410
:102474006004902F80E001E110E00E94600410E00D
:10248400802B912B8093D8239093D92303E010E0E1
:102494000E9460040093EB230CE110E00E946004AE
:1024A4000093EC2304E110E00E9460040093DE2317
:1024B40003E110E00E9460040093F62309EF11E0A9
:1024C4000E9460040093ED2307EF11E00E94600472
:1024D4000093F4230CE010E00E9460040093F523C1
:1024E4000CEF11E00E9460040093EE2302EF11E070
:1024F4000E9460040093E42306EF11E00E9460044C
:102504000093F2230DE010E00E9460040093F32393
:102514000AE010E00E946004802F90E00BE010E0DD
:102524000E946004102F00E0802B912B80930424E0
:102534009093052409E010E00E9460040093EA23CC
:102544000091EA23073040F400E01091EA231123BC
:1025540019F00060002341F001E00093EA2321E038
:1025640009E010E00E94AA040EE110E00E94600459
:102574000093E9230EEF11E00E9460040093E72327
:102584000DE110E00E9460040093E8230BE110E0E9
:102594000E9460040093FA2308EF11E00E94600493
:1025A400009360230FE110E00E9460040093E32392
:1025B40008E010E00E9460040093FF2305EF11E09F
:1025C4000E9460040093FE23E4E0F4E200810160D1
:1025D4000083899199910895E4E4F6E010811260F2
:1025E40010830E94AA01E4E4F6E000810D7F0083D9
:1025F40008959A938A9389E00091EC23801B00E06C
:1026040000931C2406E51091572311230AF44FC0AC
:1026140020915723322F330F330B10E0201731074B
:102624000CF045C04AE0009157230E94F91D402F49
:102634004A5F00910424109105240E94171E017022
:102644000023A9F50091E423013019F404E0C4DF68
:1026540005C0E4E4F6E000810260008300915723A2
:1026640007345CF0E4E6F6E0008104600083E4E60D
:10267400F6E000810D7F008357C000915723093293
:102684005CF0E4E6F6E0008102600083E4E6F6E054
:1026940000810460008348C0E4E6F6E00081026043
:1026A4000083E4E6F6E000810B7F00833DC00091E7
:1026B40057230023CAF590E00091D4231091D52329
:1026C400801791078CF584E04CEE009157230E940B
:1026D400F91D801B482F00910424109105240E94A9
:1026E400171E0170002301F50091E423013019F451
:1026F40004E072DF05C0E4E4F6E0008102600083D8
:102704000091572300235AF0E4E6F6E000810260CA
:102714000083E4E6F6E000810B7F008305C00091AE
:102724006406097F009364068991999108950E9433
:102734003A2180915523909156230196AC01652F3F
:10274400660F660B762F00E01CE62CED32E00E944B
:102754009C1E48E050E060E070E00E949C1EC801AE
:10276400D90148EE53E060E070E08C019D010E94C5
:102774009C1E08500093FB2381380EE3900700E071
:10278400A00700E0B0073CF001E00093F72302E06B
:102794000093040206C000E00093F72302E00093D4
:1027A400040208E010E020E030E0AC01BD010E942A
:1027B400491E40E750E060E070E00E949C1E0093D8
:1027C40068231093692345E00091682310916923DD
:1027D4000E94111E40E250E00E94091E00936823EB
:1027E400109369234EE750E0009168231091692308
:1027F4000E941D1E00936A2310936B23009168238B
:1028040010916923009366231093672346E150E0F7
:102814000091F72310E0401B510B009155231091B8
:1028240056230E94351E00936C2310936D23E4E01D
:102834000C944B210093DE2310912002137E1093FD
:1028440020020A95000F000F10912002102B109304
:1028540020020895D5DD6BDF2091D8233091D92350
:102864000091D6231091D723F5D0AFDD0091DE235C
:10287400E1DF0091EA232AD20091FF2310E01195B1
:1028840001951040212F220F220B322F0E94FE1E91
:1028940043E353E365E672E40E9437200E94CC27A9
:1028A400A801B90100E010E020E83FE30E943720CE
:1028B400EFE3F1E2008311832283338301E0009389
:1028C400E123089522E02093CA01F801049000E076
:1028D4000093CA01002D08959A938A9390E088E0AA
:1028E40005C0082F10E0EEDF900F83958631C8F302
:1028F400992309F493E0092F8991999108950E94ED
:102904003B210BEE11E00E9460040F3F09F047C029
:102914000CEE11E00E9460040F3F09F040C0DCDFC0
:10292400A02F07DD8091DA2320915323820F209179
:102934006223820F800F90E003C00E94D6259395F6
:102944009817D8F30E94D625802F853008F489E59E
:10295400282F0BEE11E00E94AA042A2F0CEE11E09E
:102964000E94AA0420E00DEE11E00E94AA0420E0D7
:102974000EEE11E00E94AA0420E003EF11E00E9491
:10298400AA040E94D625202F0AEE11E00E94AA0470
:102994000E94D625202F09EE11E00E94AA04E3E04C
:1029A4000C944C219C01A801CA01892F90E04F7F0F
:1029B40050708C010E94091E080F191FC801840F52
:1029C400951F0796982F80E00FEF10E0041B150B5E
:1029D400A8014F7F5070842B952B8C01C901089559
:1029E4000E943A210BEE11E00E946004B02FA0E097
:1029F4000CEE11E00E94600410E0A02BB12B0DEE50
:102A040011E00E946004902F80E00EEE11E00E941D
:102A1400600410E0802B912B8D01C4DF0817190787
:102A240081F45ADF202F30E00FEF10E08F7F907099
:102A3400081B190B2017310721F402E00093FD2332
:102A440006C000E00093FD2301E00093FD23E4E0D1
:102A54000C944B210E9434214801D90180E090E07C
:102A640046C00DE210E0AC010E94091EA801480D09
:102A7400591D483601E0500714F0485651408D0165
:102A8400212F220F220B322F0E94FE1E2801390112
:102A94008A01212F220F220B322F0E94FE1E0801D1
:102AA400190145E35AEF6EE87CE3800191010E942D
:102AB400BE1F0E948926A201B3010E94BE1F2801E5
:102AC40039018D01212F220F220B322F0E94FE1E6D
:102AD400A201B3010E945D1F0E940B1F9C01220FE3
:102AE400331FF901ED54FD4D0083118301968830A5
:102AF40000E090070CF4B5CFEAE00C9445219A93DA
:102B04008A9320E030E000E010E0A4DF08E00E94B7
:102B1400AA010091622310916323043620E0120776
:102B240008F4AFC088EE9DEF00E010E0009321248C
:102B34001093222408C0E1E2F4E2008111810D5FC8
:102B44001F4F008311830091212410912224083601
:102B540021E012072CF5209143213091442100916A
:102B640021241091222476DF03E00E94AA0100911F
:102B740062231091632308171907E8F680916223F2
:102B840090916323009121241091222400931D2409
:102B940010931E24E0916223F0916323F29758F678
:102BA40088EE9DEF00E010E0009343211093442150
:102BB40008C0E3E4F1E2008111810C5E1F4F008341
:102BC40011830091432110914421083E27E012070C
:102BD4002CF5209143213091442100911D24109122
:102BE4001E2438DF03E00E94AA01009162231091A1
:102BF40063230817190790F480916223909163234B
:102C0400009143211091442100931F241093202408
:102C1400E0916223F09163237E9758F620911F245C
:102C24003091202400911D2410911E2413DF009163
:102C34001F24109120240093D8231093D9230091AA
:102C44001D2410911E240093D6231093D723309172
:102C5400D723232F0EE010E00E94AA042091D6234C
:102C64000FE010E00E94AA043091D923232F00E141
:102C740010E00E94AA042091D82301E110E00E94F0
:102C8400AA0405E0A9DC89919991089500EB0093C9
:102C9400010202E20093020203E0009304020091A5
:102CA400F723013021F402E00093040203C003E09F
:102CB4000093040203E00093200208E2009321023F
:102CC400E0E0F2E00081016000830895013051F4F6
:102CD40001E010E800930424109305240AE0009313
:102CE400DF230895023051F40FE110E80093042427
:102CF4001093052408E00093DF230895033051F472
:102D04000FE110E8009304241093052404E00093D9
:102D1400DF230895043051F40FED10E800930424E8
:102D2400109305240AE00093DF230895053049F445
:102D34000FE510E800930424109305240AE000939F
:102D4400DF2308950E943A21F89400E30E945C0175
:102D54000091200603600093200600914006006F56
:102D64000093400600916006086300936006E0E467
:102D7400F6E0008102600083009160060660009323
:102D84006006E0E8F6E000810460008304E10E944C
:102D9400AA01E4E8F6E00081046000830AEF11E090
:102DA4000E9460040F3F09F0F5C000EF11E00E949B
:102DB40060040F3F11F481E001C080E001EF11E0F5
:102DC4000E9460040F3F11F401E001C000E0802381
:102DD400882351F020E000EF11E00E94AA0420E0D3
:102DE40001EF11E00E94AA0400E00093192405C039
:102DF4000091192403950093192400911924043097
:102E040008F0C3C000E00093182413C0FC01E65886
:102E1400FD4F24918C0100541E4F0E94AA04019678
:102E2400893000E0900790F30091182403950093F3
:102E34001824009118240330D8F622E001E010E0B1
:102E44000E94AA0428E002E010E00E94AA0420E004
:102E540005E010E00E94AA0424EB06E010E00E94C2
:102E6400AA0422E808EF11E00E94AA0420E00EE080
:102E740010E00E94AA0420E00FE010E00E94AA04DF
:102E840020E000E110E00E94AA0420E001E110E04B
:102E94000E94AA042FE003E010E00E94AA0428E0A4
:102EA4000CE110E00E94AA0421E004E110E00E9479
:102EB400AA0420E009EF11E00E94AA0425E00CE036
:102EC40010E00E94AA0421E00DE010E00E94AA0490
:102ED40022E007EF11E00E94AA0421E00AE010E0DA
:102EE4000E94AA0420E80BE010E00E94AA042FE24A
:102EF4000CEF11E00E94AA0421E009E010E00E9416
:102F0400AA0424E106EF11E00E94AA0420E00DEFD8
:102F140011E00E94AA0421E00EEF11E00E94AA042D
:102F240021E002EF11E00E94AA0427E00DE110E085
:102F34000E94AA0421E00BE110E00E94AA0421E00F
:102F44000EE110E00E94AA0420E005EF11E00E94C7
:102F5400AA0420E00AEE11E00E94AA0420E20EEF87
:102F640011E00E94AA0428E508E010E00E94AA04E7
:102F740021E003E110E00E94AA0421E00FE110E047
:102F84000E94AA0480E090E04BCF20E00AEF11E019
:102F94000E94AA0400E513EC0E94A30101E000933F
:102FA400000900915523109156230093260910938C
:102FB400270903E0009306090091A200076000932B
:102FC400A20007E00093400804ED11E000936608B6
:102FD4001093670801E0009346080E948D01009158
:102FE4009300043019F400E100932203E1E4F6E0D5
:102FF40000810860008303E00093A5080FE60093B6
:10300400A60802EF0093A70808E10093A40800E1D2
:103014000093A308E2EAF0E000810160008300E08D
:1030240000931A2400914406006F0093440602E0C2
:103034000E94AA012BDE00E210E044DC00930C02A3
:1030440001E210E03FDC00930D0202E00093220253
:103054000E9486010E947F0100E00093192400E091
:1030640000931824F7DB009164060660009364065D
:103074000091E423013011F4A3E001C0A2E080E058
:1030840090E006C00EE1A8DA0EE10E94AA010196C2
:10309400B0E08A179B07B0F300916406097F0093A0
:1030A40064069EDC78940EE10E94AA0101E000937C
:1030B400E12300E00093FC230AE00093E62300935D
:1030C400E52300E010E020E030E0E4EAF3E20083EE
:1030D400118322833383E8E9F3E20083118322839B
:1030E40033830093582301E010E0009306241093E7
:1030F400072400E00093F82308EA00935E2300937A
:103104005D2304E10E94AA013CC0E4E6F6E00081EC
:103114000260008308EA11E60E94A301E4E6F6E0F7
:1031240000810D7F008380910824909109240196E9
:103134008093082490930924853301E290070CF1CD
:1031440000E010E0009308241093092400E00093A9
:10315400A408009144060F7000934406009164068D
:10316400097F0093640601E00093F1230091622338
:1031740010916323043F21E0120718F401E0009347
:10318400E1230091EF230023E1F300E00093EF2318
:103194000091FC23013041F500E00093FC230091F1
:1031A40061230B3370F001EF11E00E94600403957A
:1031B400202F01EF11E00E94AA0400E00093612394
:1031C40005C00091612303950093612300911C24A1
:1031D400039500931C24043139F406E1FDD9E4E895
:1031E400F6E000810B7F008304E11091EB23011BC7
:1031F400009300240091E423013009F097C1E8E72B
:10320400F3E20081118122813381E0E9F3E200835A
:10321400118322833383ECE7F3E20081118122815D
:103224003381ECE9F3E20083118322833383009139
:10323400EA23053079F4E0E9F3E200811181228187
:10324400338135952795179507950093D2231093CD
:10325400D32326C0ECE9F3E200811181228133817A
:103264000E94FE1EC801D901E0E9F3E20081118148
:10327400228133810E94FE1EEFE3F1E240815181FD
:10328400628173810E94BE1FA801B9018C019D0156
:103294000E94A11F0E940B1F0093D2231093D323DB
:1032A40000910024102F110F110B2091D223309183
:1032B400D323021713070CF003C100E00093E523A6
:1032C4000091E62303950093E6230B3018F001E008
:1032D4000093E123E4E9F3E2008111812281338147
:1032E400E0E9F3E24081518162817381401B510B1B
:1032F400620B730B4083518362837383E0EAF3E2CE
:103304000081118122813381ECE9F3E24081518112
:1033140062817381401B510B620B730B4083518399
:1033240062837383E0E9F3E20081118122813381B6
:10333400E0E9F3E240815181628173810E94491E78
:10334400C801D901ECE9F3E24081518162817381C2
:10335400ECE9F3E200811181228133810E94491E4C
:10336400800F911FA21FB31F8C019D010E94FE1E9E
:103374000E9457270E940B1F1595079500930A2456
:1033840010930B2400910A2410910B24212F220F57
:10339400220B322F0E94FE1E0E9428250E940B1F22
:1033A40000935F23ECE9F3E20081118122813381F0
:1033B4000E94FE1EA801B901CA01DB01E0E9F3E2A3
:1033C40000811181228133810E94FE1EAC01BD0166
:1033D4000E9405110093572300910C2410910D2491
:1033E4002091D2233091D32302171307A4F4009120
:1033F40057230093592300910A2410910B2400931E
:103404000624109307240091D2231091D323009310
:103414000C2410930D240091572310915B23011762
:1034240024F40091572300935A2300915A230093C4
:103434005B230091592300935C230093572300914D
:103444005723075A0331F0F400915723102F110F1B
:10345400110B20915E23322F330F330B021B130BFE
:1034640044E050E00E94351E10915E23010F00934A
:103474005D2300915D2300935E2300915D230A95F3
:1034840000935D238091D2239091D32302968C01E3
:10349400212F220F220B322F0E94FE1E0E9428256C
:1034A4000E940B1F10E00093D4231093D5230091A6
:1034B400FA231091E623011708F097C19AD895C111
:1034C400E0E9F3E20081118122813381E4E9F3E24E
:1034D4000083118322833383ECE9F3E200811181B9
:1034E40022813381E0EAF3E2008311832283338370
:1034F40000E000935F2310E000930C2410930D244C
:1035040000E010E00093062410930724009358234E
:10351400009357230AE500935A2300E00093E6231F
:103524000091E52303950093E5235FC1E8E7F3E207
:103534000081118122813381E0E9F3E20083118368
:1035440022833383ECE7F3E200811181228133810A
:10355400ECE9F3E200831183228333830091EA23AD
:10356400053079F4E8ECF3E20081118122813381A2
:1035740035952795179507950093D2231093D32358
:1035840026C0ECECF3E200811181228133810E9498
:10359400FE1EC801D901E8ECF3E200811181228109
:1035A40033810E94FE1EEFE3F1E24081518162818A
:1035B40073810E94BE1FA801B9018C019D010E9464
:1035C400A11F0E940B1F0093D2231093D3230091B9
:1035D400D2231091D323212F220F220B322F0E94AA
:1035E400FE1E0E9428250E940B1F0093D4231093D3
:1035F400D52300910024102F110F110B2091D223F9
:103604003091D323021713070CF0B7C000E00093E6
:10361400E5230091E62303950093E623E4E9F3E22E
:103624000081118122813381E0E9F3E240815181FB
:1036340062817381401B510B620B730B4083518376
:1036440062837383E0EAF3E2008111812281338192
:10365400ECE9F3E24081518162817381401B510B9B
:10366400620B730B4083518362837383E0E9F3E25B
:103674000081118122813381E0E9F3E240815181AB
:10368400628173810E94491EC801D901ECE9F3E209
:103694004081518162817381ECE9F3E200811181FF
:1036A400228133810E94491E800F911FA21FB31FE4
:1036B4008C019D010E94FE1E0E9457270E940B1F31
:1036C40043E00E94171E00930A2410930B24ECE994
:1036D400F3E200811181228133810E94FE1EA80140
:1036E400B901CA01DB01E0E9F3E200811181228121
:1036F40033810E94FE1EAC01BD010E94051100939E
:10370400572300910C2410910D242091D223309141
:10371400D32302171307A4F40091572300935923CA
:1037240000910A2410910B2400930624109307247B
:103734000091D2231091D32300930C2410930D24D1
:103744000091592300935C230093572300910A248A
:1037540010910B24212F220F220B322F0E94FE1EC8
:103764000E9428250E940B1F00935F230091E623EB
:103774000B30D8F10E94FB1238C000916406097F17
:1037840000936406E4E4F6E000810D7F0083E0E941
:10379400F3E20081118122813381E4E9F3E20083C1
:1037A400118322833383ECE9F3E2008111812281C6
:1037B4003381E0EAF3E2008311832283338300E060
:1037C40010E000930C2410930D2400E010E000930B
:1037D40006241093072400935F2300E00093E6235C
:1037E4000091E52303950093E5230091E523083236
:1037F40041F010E00091E623043619F01060112323
:10380400F9F000916406097F00936406E4E4F6E0AD
:1038140000810D7F008300E010E0009306241093E4
:103824000724009358230093572300E000935F2359
:1038340010E000930A2410930B2401E00093E12389
:1038440000915723102F110F110B00930E24109386
:103854000F24809106249091072403968C01212F34
:10386400220F220B322F0E94FE1E0E94282540E0C8
:1038740050E060E87FEB0E945D1F0E940B1F0093E5
:10388400102410931124E091D223F091D32337977D
:103894002CF000910E240093582309C00091582362
:1038A400102F110F110B00930E2410930F24E0918D
:1038B400D223F091D3233B970CF4ABC04091102456
:1038C4005091112400910E2410910F240E94351E52
:1038D40042E050E00E94351E009302248091592357
:1038E400982F990F990B00915B23102F110F110B37
:1038F400801B910B03968C01212F220F220B322F58
:103904000E94FE1E0E9428250E940B1F0093122471
:103914001093132400910224102F110F110B4091C6
:103924001224509113240E94351E00930224009106
:103934000E2410910F24063520E012073CF042E0DB
:10394400009102240E94F91D0093022400910E2488
:1039540010910F248091FB2390E0C2960817190759
:103964009CF00091FB2310E0015C1F4F20910E247A
:1039740030910F24021713073CF042E00091022417
:103984000E94F91D009302241091112411231AF4AA
:1039940000E0009302240091022400231AF400E0C2
:1039A40000930224009102240B301CF00AE00093DF
:1039B400022400910224102F110F110B20913E219B
:1039C400322F330F330B021B130B42E050E00E94E3
:1039D400351E10913E21010F009302240091022410
:1039E40000933E210091022400933E2100910E2475
:1039F40010910F242091102430911124020F131FD1
:103A0400012B19F400E00093022400910224009396
:103A14000124E8E8F6E0008103FF15C00AE00E94F3
:103A2400AA01E8E8F6E0008103FF0DC000916406F6
:103A340006600093640606E10E94EE12E4E8F6E0F4
:103A440000810B7F00830091F023013039F400E002
:103A54000093F02303E00E94EE1251D80091032456
:103A6400013009F060CB00E0009303240091F123BE
:103A7400013009F04ACBE4E6F6E0008104600083FB
:103A840008EA11E60E94A301E4E6F6E000810B7F58
:103A9400008349CB00008895FECF0E943621C801DF
:103AA400D9012A013B015CD057D071F48201930102
:103AB40053D051F401E2E3E2F4E2008341830FEFD7
:103AC4001FEF2FE73FE73DC044D0A201B3010E949E
:103AD4005D1FAC01BD0140D061F442D03AD00E94D8
:103AE400D8200BED1FE029EC10F43FE32AC03FEB94
:103AF40028C0A201B3012DD00E943720080119016A
:103B04002FD0820193010E94C02023D0A0F41CD0A6
:103B140050F424D0A801B9010BED1FE029E430E4EE
:103B24000E94A11F0EC01AD04BED5FE069E470EC57
:103B34000E945D1F06C008D010F410D002C00ED041
:103B44003058E8E00C9447210E94D820800191016C
:103B540008958C019D0108950C94B6200C94ED25D4
:103B640040E050E060E070E008953F7741E00C945D
:103B74008C2603E20DBF01E20EBFC0E0D1E20E9439
:103B8400AB25002311F00E946F260E94A4160E9408
:103B94004C1D0C944C1D0D01DA0140E050E060E036
:103BA40070E00E94B62039F400E010E04D934C938D
:103BB40020E030E00CC0B901660F771F7E57572F05
:103BC400550F550B7D935C932F7730783F63D0016D
:103BD40008950024E8E0EA9532F0001F001C041662
:103BE400D0F3041AF8CF001F402D00950895FF2745
:103BF400442312F4F1604195002312F4F0950195E9
:103C04000E94EB1DF0FD0195F1FD41950895149F6F
:103C1400102D059F100D049F002D110D08954A9538
:103C24001AF016950795FBCF08954A951AF0159545
:103C34000795FBCF089500241124EFE0001F111F06
:103C4400001C111C0416150610F0041A150AEA9536
:103C5400AAF7001F111FA001009510950895519512
:103C6400419550400895FF27552312F4F160F7DF82
:103C7400112312F4F09507D00E941D1EF0FD03D00D
:103C8400F1FDEDCF0895119501951040089522247A
:103C9400349F302D259F300D169F300D079F300D1A
:103CA400249F202D310D159F200D311D069F200DC1
:103CB400311D149F102D210D321D059F100D211D46
:103CC400321D049F002D110D221D321D08954A95A9
:103CD4002AF03695279517950795F9CF08954A95B3
:103CE4002AF03595279517950795F9CF089500245F
:103CF40011241001E0E2EA9592F0001F111F221F27
:103D0400331F001C111C221C331C04161506260626
:103D1400370688F3041A150A260A370AECCF001F5F
:103D2400111F221F331FA001B1010095109520958A
:103D340030950895FF27772312F4F16015D03323CB
:103D440012F4F09509D00E94791EF69508F404D077
:103D5400F69508F409C008953095209510950195BD
:103D64001F4F2F4F3F4F0895709560955095419583
:103D74005F4F6F4F7F4F0895FF27112477FB660F26
:103D8400771F089409F4771F679517F8EE27002426
:103D940037FB220F331F089409F4331F279507F8C4
:103DA400089527FD0EC0EE0F001F111F221F3A9524
:103DB4003230B8F7332319F427FD31E002C027FF6E
:103DC40030E0E03821F400FF08940EF488940F4F9B
:103DD4001F4F2F4F3F4F323038F4332319F427FD50
:103DE40031E002C027FF30E03F3F29F0220F000CF2
:103DF400379527950895ACC0032E002012F40E9435
:103E0400AE1EE02F012F122F232F3EE9D1CF002425
:103E1400F8CFBCDF432F4F5748F04F3148F007FC31
:103E240091C03FE72FEF1FEF0FEF089533278CC0AA
:103E3400322F212F102F0E2F4F5141950E94691EB2
:103E440007FE08950C94AE1EF901EE0FFF1F37FB19
:103E5400FF3F31F0EF2BE12BE02B8894B8940895C9
:103E6400E02BE12B21F008949894B8940895989449
:103E7400889438940895FB01EE0FFF1F77FBFF3FF2
:103E840031F0EF2BE52BE42B8894B8940895E42BC0
:103E9400E52B69F3E8CFEFDF68F021F43723262F11
:103EA4008A010895372FFBCFE6DF20F00BF0089549
:103EB4007327EAF751C0C8DFE8F3B3F361F3DBDF3C
:103EC400C8F383F3A1F358DF401751076207730760
:103ED40031F4011411F10024E89488942BC078F093
:103EE400332E372F732D322E262F632D312E152F7F
:103EF400532D302E042F432D302C012C132C371727
:103F040039F0669557954795F795E0407395F7CF47
:103F1400E7FBEE0FE0E010246AF0EF0F041F151F1B
:103F2400261F60F4279517950795E79508F468947C
:103F340033953ECFEF0B040B150B260B39CFE0E87E
:103F44007E27B9CF302D30782227112700270895F6
:103F54003FE7302920E8F9CF3FEF2FEFF6CF8BDF93
:103F6400D8F3D1F370783727089585DFA8F3A3F346
:103F7400F9CF3078372793CF67DF70F383F3A9F352
:103F84007ADF50F3B3F3A9F3F7DE0124E8943F5743
:103F9400E040370FEF1F12F0D9F603C03A3E90F21B
:103FA4006894E0E00A92AA933A93AA27332422243D
:103FB4003327049FF001059FF00D712D731F149F8B
:103FC400F00D711D221C069F700D211C331C159FC2
:103FD400700D211C331E249F700D211C331E169F4F
:103FE400200C311CAA1F259F200C311CA31F269FC7
:103FF400300CA11D39915EF43395A695379427941E
:104004007795F795E79533953130BCF316C0AA231D
:1040140022F0332351F4339510C0339571F4A991F0
:10402400099096CFA7FD09C03A95EE0FFF1F771FA1
:10403400221C331CAA1F3230A8F7E894FE2B09F087
:1040440068942A2F8101E72FA9910990BACE13DF32
:1040540010F00BF087CF80CF0EDFE9F3E0F3032EEF
:10406400072670CF032E072673CFEEDEA0F37BF373
:1040740099F301DF80F39BF3A9F37EDE012427FD8E
:1040840006C0000F111F221F3150E040F8CF67FD1A
:1040940006C0440F551F661F7150F040F8CFE894D6
:1040A400371BEF0B3158EF4F2AF0EE23E9F63F3F71
:1040B400D9F203C03A3EA8F26894E0E0F0E011249B
:1040C400139440175107620738F0315008F468948C
:1040D400000F111F221FEE1F041B150B260BEF0BE5
:1040E400000F111F221FEE1F0A9279E17A95AAF0A0
:1040F400041715072607EF0730F0041B150B260BD2
:10410400EF0B089401C08894111C221C331C001C62
:10411400000F111F221FEE1FE9CFF0F9E894E22BE4
:10412400E12BE02B09F068940694379427941794B4
:10413400E79508F468947395B9F30990332311F063
:10414400F0FF09C0369427941794E79508F468940F
:1041540033953130BCF3012D122D232D32CE8BCE6D
:1041640098940895189408956FDED0F3C1F383DE14
:10417400B8F3041715072607370708957CDEA0F067
:1041840063DE90F029F0E32FE7273AF473170895DC
:1041940072DE51F04EF008940895041715072607AF
:1041A400370719F016F4B8F78894089564DEE0F33D
:1041B4004BDED0F3E7DFC0F3089408957591659161
:1041C40055914591159011FA259035900895F9DF90
:1041D400041B10E003C0F4DF041B150B20E030E0E7
:1041E40005C0ECDF041B150B260B370BB8F010FCD5
:1041F40017C045910590E00FF11F0417100540E02A
:104204002407340758F436F404910024F101E01B28
:10421400F0090994E00FF11F25903590F1010994FC
:1042240011F4D6F7F1CF31960EF0319650E060E0FC
:1042340070E045914B3F48F089F34F3F29F04E3FE2
:1042440011F07591659155914591041B150B260B41
:10425400370B39F318F3E7CFFA92EA92DA92CA925B
:10426400BA92AA929A928A927A926A925A924A92AA
:10427400BA93AA939A938A930895FF84EE84DD8473
:10428400CC84BB84AA84998488847F806E805D807A
:104294004C80BB81AA8199818881F0E0EC0FFD1FDD
:1042A400EF0108950E942E21C1D37A015B016B01B5
:1042B4008824992450D157D130F160E070E00E94F5
:1042C400B620D1F50989002309F449C08E149F044E
:1042D4004CF40CEF80160FEF900624F000E0088BEE
:1042E400E818F9080FEFE00EF01E0A890023A9F17F
:1042F40000E0098B34C027D10E94372097D30AE00D
:10430400800E00E0901E47EB53E46AEB71E52AD17E
:1043140090F325D160E271E425D1A0F60E94372004
:1043240085D301E0800E00E0901EF3CF0CD17CD346
:1043340006EF800E0FEF901E40E057EE6BED7EE22D
:1043440007D1A0F308D104D108F0BCCF60E271E436
:104354006BD30FEF800E901EF5CF01E00A8B088916
:10436400002319F06624772444C09920EAF4DDD0B0
:104374002701E0D06624772404C0D7D00FEFE00EE5
:10438400F01E4FD3861497041CF40E2D0F29A9F7A1
:104394000FEF1FEF04191509801691060CF473C072
:1043A40077246624639425C034017194619400E0F9
:1043B400700A1FC0DAD00E940B1F402E212F220F3B
:1043C400220B322F0E94FE1EA801B901CED00E94FA
:1043D400A11FA801B90100E010E020E231E424D3D8
:1043E400042D005DA3D0930101E0F6D2232B09F440
:1043F400A1D0E614F704F4F6B2D060EA70E4B2D0C7
:1044040008F041C044244394C6010197FC01008193
:104414000E3251F0040D00830A3329F400E30083C3
:104424004424439401C044240197AE16BF0670F39C
:1044340040FA4EF508890023B1F0C60102C000839A
:104444000197A816B90658F4FC0102910E32FC013A
:10445400B1F732970081FC0100830197F1CF01E0AD
:10446400800E941E0DC001E0C00ED41EC60105C00E
:10447400FC010291FC0100830197A816B906C0F360
:1044840001E3F50100830989002311F408C0C6D2B1
:10449400F60102910033D9F30E3209F4BFD2088930
:1044A4000023C1F1F601019399203AF40DE23FD0C3
:1044B4009194819400E0900A02C00BE238D0442425
:1044C40055240AE0C00ED41C01E06FD251D0405DE7
:1044D400F60141936F014CD04801012BA9F702E08A
:1044E400401600E0500684F33201820117D0208187
:1044F400830114D0E40DF51D3B9720830FEF400E8C
:10450400501E01E0401600E050067CF706EFC00E96
:104514000FEFD01E8601E3E10C943F211195019524
:104524001040F601E00FF11F089500E3F601019336
:104534006F0108950E2D0F2919F40A89002311F033
:104544000EE2F5DF089549EF52E065E170E5089564
:104554000CD00C94C02003D060E87FE3089540E0C1
:1045640050E0089502D00C94D8208C019D01089548
:104574004AE050E084010C94351E0E942E21EF97EE
:10458400EF976A972A873B874887598768017B0199
:1045940000E00D830E8302C005D20ED229D205326B
:1045A40049F00023C9F70D811E81EF96EF966A96B4
:1045B400E0E1B2CF0081053221F42BD2F3D105E240
:1045C400ECCF00E00C830B830A8309833E0102E1F4
:1045D40003D205E411E2088B198B06C0098100237C
:1045E40011F40081098315D2FBD10052B9F30350B1
:1045F40059F00850B1F3025019F0035049F00CC0BF
:104604000A8103950A83EFCF0B8103950B83EBCFCC
:104614000C8103950C83E7CF00810A3279F4B6D17B
:10462400AD90BD90AFD1BB203AF4B194A19400E019
:10463400B00A0A8103950A83ECD114C0AA24BB24CE
:104644004AE050E00DC021916F0185010E94091ECE
:10465400A22EBB24A00EB11E00EDA00E0FEFB01EC3
:10466400C2D188F30A81002311F000E00C83B8D191
:104674000E32F1F4CED1B4D10A3231F487D18D9017
:104684009D9080D1C6D117C0882499244AE050E077
:10469400AAD188F421916F0184010E94091E822EFF
:1046A4009924800E911E00ED800E0FEF901EF0CF26
:1046B40088248A94982C80E093D10C5421F00C51D6
:1046C40031F0045039F481E0C80EA5D103C001E0F3
:1046D400C00ED81E8DD1E4E8F2E00C94E92080FBF2
:1046E4005EF44D815E81652F660F660B53D1408366
:1046F40051836283638352CF2D813E814BD12083CA
:1047040031834CCF43D10D9111963CD10A8B2E01AC
:1047140003E14BD1FAC03AD16D907D9033D1062D8F
:10472400072921F406E5602E01E2702E992022F477
:1047340000E1802E07E2902E80E090E001C0019617
:10474400F30101913F01002319F088159905BCF389
:1047540068D12301919581959040680E791ED5C04A
:104764000B81002331F0082D092919F49924882498
:10477400839405E611E2088B198B0881003739F41C
:1047840005D1F6D000E122D100E009832BC0FDD091
:104794001EF4F4D04BD101C0EBD008810F3611F4D4
:1047A40008E0F1CF053771F70AE0EDCFEED04D9177
:1047B4005D9126F46D917D91E5D005C0E3D0652F20
:1047C400660F660B762FCA01DB0177234AF40DE2EC
:1047D40009839095A095B09581959F4FAF4FBF4F9A
:1047E4000AE0F4D03E0107E9F7D02E0107E9DDD055
:1047F400082F092B0A2B0B2B11F001E001C000E05C
:104804000F83082D092919F40F8100FF17C0FAD06E
:10481400E889F989E00DF11D0081F30102933F015C
:10482400F1D004D1012B022B032B89F7992032F408
:104834000C81002319F0FDD001C0DFD08E01095690
:104844001F4F91D0D4F30B81002309F45EC00F8174
:1048540000FF5BC00881083711F0083549F4E1D046
:10486400F30108810083DDD000E3F30100834DC030
:104874000F3609F04AC0F3010081003309F445C042
:1048840000E302933F0141C081E0088102500883A4
:10489400082D092939F499248824839408C000E058
:1048A400088380E099201AF406E0802E99246ED0C3
:1048B40065D055DE60E070E00E94C02028F44DE22F
:1048C4004983732F7058372F3E0142E1640E751EE1
:1048D4006A0C7B1C4B814A938A934A814A93B301A5
:1048E400A401E0DC28010C81002379F0A2D082012C
:1048F4003AD05CF482D0FBCF91D006E7602E01E27F
:10490400702E09E7402E01E2502E420186189708C6
:10491400A814B9041CF480E090E007C090D0A81853
:10492400B90810E0A01AB10AC5010A81002321F4D4
:1049340001C03FD00197EAF70981002339F032D052
:1049440004C030D0F30101913F0136D00FEF800E47
:10495400901EBAF70A81002309F420CE01970AF4C5
:104964001DCE27D0FBCF0619170908151905089580
:104974008D919D9107D0A0E0B0E008950D911D9117
:104984002D913D91A083B183089580FBF701A0810F
:10499400B1810895F701A081B1810D911D91F2DFDC
:1049A400F8010895288539850895400E00E0501EC9
:1049B40008952885398500E2EA85FB8509950D81EE
:1049C4001E810F5F1F4F0D831E83089510E00C8717
:1049D4001D871E871F870895600E00E0701E0895CE
:1049E400F60100810895F601008100530A3008950C
:1049F400F60101916F010883089500E3F301029326
:104A04003F0108954C855D856E857F85AEDD0C94F0
:104A1400791E01E0C00E00E0D01E08950FEFC00E15
:104A2400FBCF0FEF600EDACF0E94BE1FC801D90181
:104A3400089505D010E04501801A910A089509816E
:104A4400002311F001E0089500E008950E9432214E
:104A5400229741E050E060E070E00E94C02060F4E2
:104A640040E00E94B62021F402E26BD03FEF5FC029
:104A740001E267D03FE75BC0AE010E94CD1DC801D3
:104A8400D90143EF54E065E37FE30E94C02068F45A
:104A940037FBAA0FBB1FB395B695A795B7F9088145
:104AA4001981015010400883198340E050E060E808
:104AB4007FEB43D02801390140E050E060E87FE318
:104AC4003CD0A801B901820193010E943720C8019A
:104AD400D901A801B9012FD0280139010881102F6B
:104AE400110F110B212F312F0E94FE1E48E152E7B6
:104AF40061E37FE320D04801590142E252E964EDC9
:104B04007EE38201930117D04DED5BE96AE27FE316
:104B140016D0A201B3010FD044E050E060E070E48D
:104B24000ED0AC01BD0107D0A401B50108D0229676
:104B3400ECE00C9443210C94BE1F8C019D010C9459
:104B44005D1FE3E2F4E2008351830FEF1FEF2FE7D1
:104B5400089501E008950E943A21C801D9011A017B
:104B64003F7740E856E968E17BE40E94D82038F4B6
:104B740016D0B38300E010E020E030E00DC03B2FFE
:104B84000E940B1F0E94FE1E0AD03383A801B901A4
:104B94008C019D010E94A11FE4E00C944B21F101C2
:104BA40000831183228308954DE65EE466EC71E48C
:104BB400EAE7F1E200811181228133810E94491EDA
:104BC400075C1F4C2F4F3F4F008311832283338395
:104BD40089011F7708950E942E21C801D901BF774A
:104BE40041E050E060E87FE33B2F0E94C02070F476
:104BF40040E00E94B62029F40BED1FE029E43FE3D6
:104C040050C0CC24DD24EE24FF241CC00BEDC02EA8
:104C14000FE0D02E09E4E02EF72E40E07FEB082FC2
:104C240048D02801390140E050E060E87FE38C017E
:104C34009D013FD0A801B901820193010E94372050
:104C4400C801D901AC01BD018C019D012DD0280101
:104C5400390144E25FEF6BE27CEB26D048E854E490
:104C640066EA7EE328D048E150EC6FE370E423D099
:104C740045EB1CD0480159014AEE54EB66E870E458
:104C84008201930118D046EB11D0A801B901840127
:104C940095010E943720AC01BD0106D0A601B701E1
:104CA40008D0E0E10C943F210C94BE1F5DEF68E650
:104CB40070E40C945D1FFDDFA201B301F5CF20E089
:104CC40006D0E9F70895259102D0E9F708952D93C8
:104CD40001501040202F212B089586EA90E5FC0115
:104CE40005911491FC013296A591B491FC0134967E
:104CF40025913491422F432B19F0F901E4DF01C0CF
:104D0400DEDF069610E5823B910748F3089540E004
:104D14000C948C260E9436212897802FB32F442E82
:104D240040E050E060E070E00E94C02010F401E038
:104D340001C000E0000F400EBF7743E859EF62E284
:104D44007FE3082F3B2F80D076D041E05CEF6FE704
:104D540077E40E94D82088F5AE010E94AD256BD07F
:104D6400042D10E06BD0488159816A817B8172D017
:104D7400088319832A833B83AE014C5F5F4F2A016A
:104D840040E050E060E87EE35FD0A2010E94AD25E0
:104D940040E050E060E870E40C811D812E813F8189
:104DA40053D0A801B901088119812A813B810E944D
:104DB400A11F0E940B1F402E0CC00E940B1F602ECF
:104DC4003DD0A801B9018C019D0133D0460C03E00C
:104DD400402240FA3EF4AC01BD0100E010E020E8BE
:104DE4003FE327D002E0401608F0B0588C019D0143
:104DF40029D0280139014BEF57ED6EE179E324D036
:104E040045E656E269E97BEB21D048E554E363EAE1
:104E14007DE31CD041EE5DE565E27FEB17D04BED01
:104E24005FE069EC7FE316D00DD02896E8E00C949F
:104E340047210E94A11FC801D901089520E030E054
:104E44000C94091FAC01BD010C94BE1F03D0A20138
:104E5400B301FACF0C945D1F1B2F6A2FF901A081B7
:104E6400B181AD014F5F5F4F408351830C93A62FF7
:104E7400B12F0895BA93AA9324970A831B838901B7
:104E84009E012A5F3F4F28833983BE01AE014E5FE6
:104E94005F4F2EE237E20E94BF2220E0AA81BB814D
:104EA4002C932496A991B99108950E9432212297B6
:104EB4004801590141E050E060E070E00E94C020E8
:104EC40098F440E00E94B62029F400E010E020E0CD
:104ED40030E04EC001E2E3E2F4E2008351830FEFDD
:104EE4001FEF2FE73FE744C0AE010E94CD1DC8016C
:104EF400D90145EC53E062E47FE30E945D1F4AE17F
:104F040051E562E17FE33BD0A801B9018C019D0129
:104F14003BD0402E088100FF14C00A952DD0802F6D
:104F240043EF54E065EB7FE3042D0E94BE1F37FB83
:104F3400220F331F380F3695279537F9C801D90149
:104F44000BC01AD0842D912FD90137FBAA0FBB1F98
:104F5400B00FB695A795B7F940E050E060E87EE35E
:104F64008C019D010CD0AC01BD01840195010CD0D4
:104F74002296ECE00C94432142E00C94F91D0E942B
:104F8400BE1F2801390108950E943720A201B301F0
:104F94000C945D1F0E9434212497B32F992440E080
:104FA40050E060E070E00E94C020882408F48394FC
:104FB400BF7743E859EF62EA7FE33B2F62D0AE014B
:104FC4000E94AD256BD080FA442440F801E04026CD
:104FD40053D00E940B1F03700A9529F00A9531F0F3
:104FE4000A9531F007C04FD0939404C0842CFCCFB1
:104FF4004AD0842CAC01BD018C019D0142D00883B0
:1050040019832A833B8344E556E768E471EC39D07D
:1050140040E759ED63E52DD0280139014DE354ED06
:105024006EE872EC29D00E945D1F488159816A8123
:105034007B8127D045E15EED66E81BD0A801B9016C
:10504400820193010E943720AC01BD011AD026D001
:1050540090FA36F4A801B9011CD00E9437201ED062
:1050640080FA0EF4B0588C019D012496EAE00C9469
:10507400452173E40C945D1F088119812A813B81C9
:1050840008950C94BE1FAC01BD0103D00E94A11F62
:1050940005C000E010E020E83FE30895C801D9010D
:1050A40008955A002421B250A7027E210000253021
:1050B40035640025303566002530336400253033EF
:1050C4006420002530345800010AD7A3BC2C0130D9
:1050D400313233343536373839414243444546005A
:1050E400286E756C6C20706F696E7465722900305F
:1050F400313233343536373839616263646566007A
:085104003F3F3F0001000000E5
:0400000300000000F9
:00000001FF
